S01800006275696C642F6D696361322F6D61696E2E737265632D
S11300000C9446000C9463000C9463000C946300FD
S11300100C9463000C9463000C9463000C946300D0
S11300200C9463000C9463000C9463000C946300C0
S11300300C9463000C9463000C9463000C9497017B
S11300400C9463000C9463000C9463000C946300A0
S11300500C9463000C9463000C9463000C94630090
S11300600C9463000C9463000C9463000C94630080
S11300700C9463000C9463000C9463000C94630070
S11300800C9463000C9463000C94630011241FBE51
S1130090CFEFD0E1DEBFCDBF11E0A0E0B1E0E0E3FF
S11300A0F6E000E00BBF02C007900D92A230B1074A
S11300B0D9F711E0A2E0B1E001C01D92AF32B1075F
S11300C0E1F70C94B7000C94000026EE80912A010D
S11300D090912B01A0912C01B0912D010097A105C5
S11300E0B10589F080FF0FC080911E0190911F011E
S11300F0A0912001B0912101863E9105A105B10591
S113010014F420911E018FB7F894992720932601A7
S113011021BF109224018FBF0E9485010895AC0174
S11301208FB7F894282F3327E0912301809123017E
S11301308F5F809323018091230187708093230133
S11301409091230180911801981759F02FBFFF2730
S1130150EE0FFF1FE95FFE4F4083518381E090E083
S11301600895E09323012FBF80E090E00895CFEF3E
S1130170D0E1DEBFCDBFD29AD09AD19AD698A79AB1
S1130180A69AA59AA49AA39AA29AA19AA09A8C9A9A
S11301908F9A8E9ABB98BF98D498DC98D39A8B9AEE
S11301A08D9ADB9ADA9AD89AD99A83E08C5F873948
S11301B0E8F360E08AE08093040160932301609394
S11301C0180110922A0110922B0110922C01109206
S11301D02D01609324018FEF80932E0180930201FF
S11301E060930501862F8D5F8093250196EE909391
S11301F026018FB7F894282F332787B78E7F87BFC0
S113020087B78D7F87BF80B7886080BF8BE083BF4F
S113021062BF91BF87B7826087BF2FBF8FB7F89443
S1130220992760932801DA9AD89AD99A8FBF609354
S113023029018DE491E0A0E0B0E080931A0190934D
S11302401B01A0931C01B0931D01609319018FB78A
S1130250F894C82FDD2782B7282F33274427552742
S1130260235B3E4F4F4F5F4F20931E0130931F017E
S1130270409320015093210181E090E0A0E0B0E0A0
S113028080932A0190932B01A0932C01B0932D010C
S1130290263E31054105510528F42093260121BF4E
S11302A00E948501CFBF7894909118018091230119
S11302B0981719F480E090E01FC08FB7F894282FA6
S11302C0332790911801809118018F5F8093180152
S11302D080911801877080931801E92FFF27EE0F92
S11302E0FF1FE95FFE4F80819181108211822FBF31
S11302F0FC01099581E090E08823B1F685B780621E
S113030085BF889500000000CFCF8091000188232D
S113031029F48EE592E00E948F0006C085B7837EA3
S113032085BF85B7806285BF80E090E008957894AA
S11303301F920F920FB60F9211242F933F934F9356
S11303405F936F937F938F939F93AF93BF93EF9339
S1130350FF938FB7F894282F3327809106018823C1
S113036069F08091220180932701886080932201A3
S113037083BF8091170181BF109206012FBF8AEDC0
S113038091E00E948F00FF91EF91BF91AF919F91F7
S11303908F917F916F915F914F913F912F910F902A
S11303A00FBE0F901F9018958FBF08958FB7F894C4
S11303B099270895CF93DF9381E08093240180915E
S11303C02A0190912B01A0912C01B0912D0100974D
S11303D0A105B10509F46DC0FD01EC0180FF69C000
S11303E08091260199270196AA2797FDA095BA2FF7
S11303F020911E0130911F01409120015091210153
S1130400281B390B4A0B5B0B20931E0130931F01F1
S113041040932001509321012330310541055105BA
S11304200CF047C0809119018823A9F480911A0126
S113043090911B01A0911C01B0911D01280F391F3F
S11304404A1F5B1F20931E0130931F01409320011C
S11304505093210114C081E090E080959095AA27E3
S113046097FDA095BA2F8C239D23AE23BF238093A1
S11304702A0190932B01A0932C01B0932D0180911C
S11304802E01882319F48FEF80932E0190912E0171
S11304909F5F90932E01809105018F5F80930501EA
S11304A0E92FFF27ED5FFE4F108286E992E00E945C
S11304B08F000E946500DF91CF91089587B7992737
S11304C08C7F009719F080E090E01AC06F9918C0F3
S11304D0379B03C088E090E013C087B799278370E7
S11304E09070892B59F081B792B7891B803118F429
S11304F08CE190E005C088E190E002C080E190E0EA
S1130500382F25B7237E8C3121F0883111F008C0B3
S1130510000080B7992787709070892BC9F7237ED4
S1130520232B25BF85B7806285BF0895909105016F
S1130530992319F461E070E016C0809102018823C8
S113054019F48FEF80930201809102018F5F8093F1
S11305500201915090930501E82FFF27ED5FFE4FB4
S11305608081682F7727662309F061C050912901A3
S11305705523F9F48FB7F894282F3327DA989091FC
S113058028019160909328012FBF8FB7F894282FEA
S11305903327D99A892F8D7F809328012FBF8FB756
S11305A0F894282F3327D89A997F909328012FBF46
S11305B01DC0409128015130E9F48FB7F894992770
S11305C0DA9A242F2E7F209328018FBF8FB7F894B7
S11305D09927D9982260209328018FBF8FB7F89468
S11305E09927D89A2B7F209328018FBF5F5F509360
S11305F0290108958FB7F894282F3327DA9A842F86
S11306008E7F809328012FBF8FB7F8949927D99AAA
S1130610242F2C7F209328018FBF8FB7F89499271C
S1130620D8982460209328018FBF609329010895EE
S10506300100C3
S9030000FC
